:020000040000FA
:040800002BEF09F0E1
:1008100003B26DEF05F0F2B48BEF05F09EB093EFED
:1008200005F09EB29BEF05F0F2A81AEF04F0F2B2C9
:100830001CEF04F0DAEF08F0CD90F2929EA026EFC4
:1008400004F00101533F26EF04F0542BAEC1B2F186
:10085000AFC1B3F1B0C1B4F1B1C1B5F1AAC1AEF14C
:10086000ABC1AFF1ACC1B0F1ADC1B1F1A6C1AAF15C
:10087000A7C1ABF1A8C1ACF1A9C1ADF1A2C1A6F16C
:10088000A3C1A7F1A4C1A8F1A5C1A9F19EC1A2F17C
:100890009FC1A3F1A0C1A4F1A1C1A5F19AC19EF18C
:1008A0009BC19FF19CC1A0F19DC1A1F196C19AF19C
:1008B00097C19BF198C19CF199C19DF1CECF96F162
:1008C000CFCF97F153C198F154C199F1CF6ACE6A55
:1008D0000101536B546B9E90CD800FBC0F8E0FBAED
:1008E00075EF04F00F8ADAEF08F00F8C0FBEB1EF4E
:1008F00004F096C19AF197C19BF198C19CF199C1FE
:100900009DF19AC19EF19BC19FF19CC1A0F19DC137
:10091000A1F19EC1A2F19FC1A3F1A0C1A4F1A1C107
:10092000A5F1A2C1A6F1A3C1A7F1A4C1A8F1A5C1D7
:10093000A9F1A6C1AAF1A7C1ABF1A8C1ACF1A9C1A7
:10094000ADF1AAC1AEF1ABC1AFF1ACC1B0F1ADC177
:10095000B1F1AEC1B2F1AFC1B3F1B0C1B4F1B1C147
:10096000B5F101015E6B5F6B606B616B96515E2749
:1009700097515F2398516023995161239A515E27C3
:100980009B515F239C5160239D5161239E515E27A3
:100990009F515F23A0516023A1516123A2515E2783
:1009A000A3515F23A4516023A5516123A6515E2763
:1009B000A7515F23A8516023A9516123AA515E2743
:1009C000AB515F23AC516023AD516123AE515E2723
:1009D000AF515F23B0516023B1516123B2515E2703
:1009E000B3515F23B4516023B5516123D890010105
:1009F000613360335F335E33D8900101613360331C
:100A00005F335E33D8900101613360335F335E330F
:100A100000C10CF101C10DF102C10EF103C10FF1D2
:100A200004C110F105C111F106C112F107C113F1A2
:100A300008C114F109C115F10AC116F10BC117F172
:100A400034C135F111B830EF05F00101620E046FC9
:100A5000010E056F000E066F000E076F39EF05F0EF
:100A60000101A70E046F020E056F000E066F000E47
:100A7000076F5EC100F15FC101F160C102F161C1A8
:100A800003F12FEC1FF003BF04D019BE02D019A050
:100A9000108C11A051EF05F010BA51EF05F00F8046
:100AA000108A0CC100F10DC101F10EC102F10FC19C
:100AB00003F110C104F111C105F112C106F113C116
:100AC00007F114C108F115C109F116C10AF117C1E6
:100AD0000BF135C134F1DAEF08F00392ABB2AB9809
:100AE000AB88030103EE00F080517F0BE92604C0C0
:100AF000EFFF802B8151805D700BD8A48B820000AA
:100B00008051815D700BD8A48B9281518019D8B42B
:100B10000790DAEF08F0F2940101453FDAEF08F0B0
:100B2000462BDAEF08F09E900101533FDAEF08F010
:100B3000542BDAEF08F09E9211B80AEF07F08BB44D
:100B4000A9EF05F010ACA9EF05F08B84109CAAEF7B
:100B500005F08B94C3CF55F1C4CF56F1C28207B4D0
:100B600014EF06F047C14BF148C14CF149C14DF1BA
:100B70004AC14EF15EC162F15FC163F160C164F1CF
:100B800061C165F196C1B6F197C1B7F198C1B8F1ED
:100B900099C1B9F19AC1BAF19BC1BBF19CC1BCF139
:100BA0009DC1BDF19EC1BEF19FC1BFF1A0C1C0F109
:100BB000A1C1C1F1A2C1C2F1A3C1C3F1A4C1C4F1D9
:100BC000A5C1C5F1A6C1C6F1A7C1C7F1A8C1C8F1A9
:100BD000A9C1C9F1AAC1CAF1ABC1CBF1ACC1CCF179
:100BE000ADC1CDF1AEC1CEF1AFC1CFF1B0C1D0F149
:100BF000B1C1D1F1B2C1D2F1B3C1D3F1B4C1D4F119
:100C0000B5C1D5F1010155515B2756515C23E86A06
:100C10005D230E2E14EF06F05CC157F15DC158F153
:100C20005B6B5C6B5D6B078E0201002FDAEF08F0E7
:100C30003C0E006F1A50E00BE00AE866128818BEFE
:100C400002D018B4108E00C10CF101C10DF102C127
:100C50000EF103C10FF104C110F105C111F106C17C
:100C600012F107C113F108C114F109C115F10AC14C
:100C700016F10BC117F134C135F101018A6748EF54
:100C800006F08B6748EF06F08C6748EF06F08D673B
:100C90004CEF06F07CEF06F08EC100F18FC101F140
:100CA00090C102F191C103F10101010E046F000E28
:100CB000056F000E066F000E076F2FEC1FF000C1CE
:100CC0008EF101C18FF102C190F103C191F1006772
:100CD00071EF06F0016771EF06F0026771EF06F041
:100CE00003677CEF06F08AC18EF18BC18FF18CC156
:100CF00090F18DC191F10F80D57ED5BE6DD0D6CF4C
:100D000047F1D7CF48F145C149F1E86AE8CF4AF148
:100D100019BE02D019A0108C109047C100F148C133
:100D200001F149C102F14AC103F101010A0E046F48
:100D3000000E056F000E066F000E076F2FEC1FF000
:100D400003AF1080010154A7B2EF06F00F9A0F9C79
:100D50000F9E0101000E5E6F600E5F6F3D0E606FB3
:100D6000080E616F010147BFC2EF06F04867C2EF8E
:100D700006F04967C2EF06F04A67C2EF06F0F28854
:100D8000E7EF06F0F2985E6B5F6B606B616B966BE2
:100D9000976B986B996B9A6B9B6B9C6B9D6B9E6B27
:100DA0009F6BA06BA16BA26BA36BA46BA56BA66BD7
:100DB000A76BA86BA96BAA6BAB6BAC6BAD6BAE6B87
:100DC000AF6BB06BB16BB26BB36BB46BB56BD76A17
:100DD000D66A0101456B466B0CC100F10DC101F1F2
:100DE0000EC102F10FC103F110C104F111C105F1EF
:100DF00012C106F113C107F114C108F115C109F1BF
:100E000016C10AF117C10BF135C134F1DAEF08F060
:100E1000DAEF08F00201002F63EF08F0D59ED6CF7D
:100E200047F1D7CF48F145C149F1E86AE8CF4AF127
:100E3000D76AD66A0101456B466BD58E1A50E00B16
:100E4000E00AE866128818BE02D018B4108E17AEF9
:100E50001C8C00C10CF101C10DF102C10EF103C1E6
:100E60000FF104C110F105C111F106C112F107C162
:100E700013F108C114F109C115F10AC116F10BC132
:100E800017F134C135F10FA0109A11B853EF07F0E4
:100E90000101620E046F010E056F000E066F000E59
:100EA000076F5CEF07F00101A70E046F020E056FDC
:100EB000000E066F000E076F47C100F148C101F137
:100EC00049C102F14AC103F12FEC1FF003BF6FEFDC
:100ED00007F019BE02D019A0108C11B00F800CC100
:100EE00000F10DC101F10EC102F10FC103F110C1FA
:100EF00004F111C105F112C106F113C107F114C1CA
:100F000008F115C109F116C10AF117C10BF135C17C
:100F100034F102013C0E006F00C10CF101C10DF172
:100F200002C10EF103C10FF104C110F105C111F1AD
:100F300006C112F107C113F108C114F109C115F17D
:100F40000AC116F10BC117F134C135F101018A67ED
:100F5000B1EF07F08B67B1EF07F08C67B1EF07F0E7
:100F60008D67B5EF07F0E5EF07F08EC100F18FC197
:100F700001F190C102F191C103F10101010E046F71
:100F8000000E056F000E066F000E076F2FEC1FF0AE
:100F900000C18EF101C18FF102C190F103C191F145
:100FA0000067DAEF07F00167DAEF07F00267DAEFC0
:100FB00007F00367E5EF07F08AC18EF18BC18FF16F
:100FC0008CC190F18DC191F10F80109047C100F15B
:100FD00048C101F149C102F14AC103F101010A0E00
:100FE000046F000E056F000E066F000E076F2FECEA
:100FF0001FF003AF1080010154A70BEF08F00F9A08
:101000000F9C0F9E0101000E5E6F600E5F6F3D0E24
:10101000606F080E616F47C100F148C101F149C11D
:1010200002F14AC103F10101140E046F050E056FB0
:10103000000E066F000E076F2FEC1FF003AF24EFBA
:1010400008F0F28849EF08F0F2985E6B5F6B606B16
:10105000616B966B976B986B996B9A6B9B6B9C6BA8
:101060009D6B9E6B9F6BA06BA16BA26BA36BA46B24
:10107000A56BA66BA76BA86BA96BAA6BAB6BAC6BD4
:10108000AD6BAE6BAF6BB06BB16BB26BB36BB46B84
:10109000B56B0CC100F10DC101F10EC102F10FC120
:1010A00003F110C104F111C105F112C106F113C120
:1010B00007F114C108F115C109F116C10AF117C1F0
:1010C0000BF135C134F18BB46DEF08F010AC6DEF5E
:1010D00008F08B84109C6EEF08F08B94C3CF55F111
:1010E000C4CF56F1C28207B4D8EF08F047C14BF124
:1010F00048C14CF149C14DF14AC14EF15EC162F1A6
:101100005FC163F160C164F161C165F196C1B6F17F
:1011100097C1B7F198C1B8F199C1B9F19AC1BAF1C3
:101120009BC1BBF19CC1BCF19DC1BDF19EC1BEF193
:101130009FC1BFF1A0C1C0F1A1C1C1F1A2C1C2F163
:10114000A3C1C3F1A4C1C4F1A5C1C5F1A6C1C6F133
:10115000A7C1C7F1A8C1C8F1A9C1C9F1AAC1CAF103
:10116000ABC1CBF1ACC1CCF1ADC1CDF1AEC1CEF1D3
:10117000AFC1CFF1B0C1D0F1B1C1D1F1B2C1D2F1A3
:10118000B3C1D3F1B4C1D4F1B5C1D5F10101555109
:101190005B2756515C23E86A5D230E2ED8EF08F0DA
:1011A0005CC157F15DC158F15B6B5C6B5D6B078E89
:1011B000DAEF08F002C0E0FF005001C0D8FF1000D5
:1011C000A6B2E0EF08F00CC0A9FF0BC0A8FFA69ED6
:1011D000A69CA684F29E550EA76EAA0EA76EA682A6
:1011E000F28EA694A6B2F2EF08F00C2A1200A96EB5
:1011F000A69EA69CA680A8500C2A120004012C0EC4
:10120000826F2AEC0BF02AEC20F00C50F7EC08F07F
:10121000E8CF00F10C50F7EC08F0E8CF01F101AF96
:1012200017EF09F00101FF0E026FFF0E036FCDEC07
:101230001FF0296723EF09F00401200E826F2AECCA
:101240000BF028EF09F004012D0E826F2AEC0BF051
:10125000D7EC1DF01200306A076A0F6A106A116A33
:10126000126A136A0F010E0EC16E860EC06E030E57
:10127000C26E0F01896A190E926E080E8A6EF10E07
:10128000936E8B6A980E946EF18EFC0EF7EC08F05C
:10129000E8CF0BF00BA011800BA211820BA41184DC
:1012A0000BA81188C90EF7EC08F0E8CF17F0CA0EAA
:1012B000F7EC08F0E8CF18F0CB0EF7EC08F0E8CF29
:1012C00019F0CC0EF7EC08F0E8CF1AF0CD0EF7ECE1
:1012D00008F0E8CF2FF01C6A1D6A0E6A01015B6BF3
:1012E0005C6B5D6B576B586BF29A0101476B486BF7
:1012F000496B4A6B4B6B4C6B4D6B4E6B4F6B506B32
:10130000516B526B456B466BD76AD66A0F01280E3C
:10131000D56EF28A9D90B00ECD6E01015E6B5F6B53
:10132000606B616B626B636B646B656B666B676B49
:10133000686B696B536B546BCF6ACE6A0F9A0F9CC4
:101340000F9E9D80760ECA6E9D8202013C0E006F3C
:10135000CC6A160EF7EC08F0E8CF00F1170EF7ECA8
:1013600008F0E8CF01F1180EF7EC08F0E8CF02F131
:10137000190EF7EC08F0E8CF03F1010103AFDBEF42
:1013800009F02AEC20F0160E0C6E00C10BF0E0EC18
:1013900008F0170E0C6E01C10BF0E0EC08F0180E0F
:1013A0000C6E02C10BF0E0EC08F0190E0C6E03C1DC
:1013B0000BF0E0EC08F000C18AF101C18BF102C131
:1013C0008CF103C18DF100C18EF101C18FF102C119
:1013D00090F103C191F11A0EF7EC08F0E8CF00F19B
:1013E0001B0EF7EC08F0E8CF01F11C0EF7EC08F04B
:1013F000E8CF02F11D0EF7EC08F0E8CF03F1010190
:1014000003AF31EF0AF02AEC20F01A0E0C6E00C187
:101410000BF0E0EC08F01B0E0C6E01C10BF0E0ECE1
:1014200008F01C0E0C6E02C10BF0E0EC08F01D0E73
:101430000C6E03C10BF0E0EC08F01A0EF7EC08F0AC
:10144000E8CF00F11B0EF7EC08F0E8CF01F11C0E1D
:10145000F7EC08F0E8CF02F11D0EF7EC08F0E8CF4A
:1014600003F100C192F101C193F102C194F103C1F2
:1014700095F1240EAC6E900EAB6E240EAC6E080E81
:10148000B86E80B662EF0AF01E0EF7EC08F0E8CFF7
:1014900000F11F0EF7EC08F0E8CF01F100C1E8FF02
:1014A000FF0A10E001C1E8FFFF0A0CE01E0EF7EC96
:1014B00008F0E8CFAFFF1F0EF7EC08F0E8CFB0FF61
:1014C00066EF0AF0000EB06E1F0EAF6E0401806B67
:1014D000816B0F01900EAB6E0F019D8A0301806B33
:1014E000816BC26B8B9207900001F28EF28C07B079
:1014F00085EF1CF00FB019EF16F010BE19EF16F0C3
:1015000012B819EF16F00301805181197F0BD8B47E
:1015100085EF1CF013EE00F081517F0BE126812B4B
:10152000E7CFE8FFE00BD8B485EF1CF023EE82F0A4
:10153000C2513F0BD926E7CFDFFFC22BDF50780A1D
:10154000D8A485EF1CF007808EC100F18FC101F196
:1015500090C102F191C103F10101040E046F000E6C
:10156000056F000E066F000E076F2FEC1FF000AF27
:10157000C3EF0AF00101030E8E6F000E8F6F000E95
:10158000906F000E916F03018251720AD8B4FDEF83
:1015900015F08251520AD8B4FDEF15F08251750A48
:1015A000D8B4FDEF15F08251630AD8B43FEF19F0BB
:1015B0008251690AD8B4ACEF12F082517A0AD8B4D9
:1015C000BFEF13F08251490AD8B44BEF12F08251A9
:1015D000500AD8B469EF11F08251700AD8B4ACEF58
:1015E00011F08251540AD8B4D7EF11F08251740A25
:1015F000D8B41DEF12F08251410AD8B440EF0CF07C
:1016000082514B0AD8B43EEF0BF082516D0AD8B428
:1016100073EF10F082514D0AD8B48CEF10F0825164
:10162000730AD8B42DEF15F08251530AD8B492EF53
:1016300015F08251620AD8B41BEF11F08251420AB0
:10164000D8B456EF11F08251590AD8B4C4EF0FF054
:1016500076EF19F0040114EE00F080517F0BE126C3
:1016600082C4E7FF802B120004010D0E826F2AEC6A
:101670000BF00A0E826F2AEC0BF0120004014B0EE5
:10168000826F2AEC0BF004012C0E826F2AEC0BF017
:1016900081B802D02FB630D003018351430AD8B4A9
:1016A00083EF0BF003018351630AD8B485EF0BF08D
:1016B00003018351520AD8B487EF0BF00301835121
:1016C000720AD8B489EF0BF003018351470AD8B4EA
:1016D0008BEF0BF003018351670AD8B48DEF0BF049
:1016E00003018351540AD8B48FEF0BF003018351E7
:1016F000740AD8B4FEEF0BF003018351550AD8B435
:1017000091EF0BF082D02F807AD02F9078D02F825B
:1017100076D02F9274D02F8472D02F9470D02F86D1
:101720006ED084C330F185C331F186C332F187C3F3
:1017300033F10101296B78EC20F0EFEC1FF000C1D0
:1017400004F101C105F102C106F103C107F16BEC1F
:1017500020F0200EF86EF76AF66A0900F5CF2CF13A
:101760000900F5CF2DF10900F5CF2EF10900F5CFD5
:101770002FF10900F5CF30F10900F5CF31F1090063
:10178000F5CF32F10900F5CF33F10101296B78EC87
:1017900020F0EFEC1FF02FEC1FF00067D7EF0BF0FD
:1017A0000167D7EF0BF00267D7EF0BF0036701D0AB
:1017B00025D004014E0E826F2AEC0BF004016F0E4F
:1017C000826F2AEC0BF004014D0E826F2AEC0BF0B5
:1017D0000401610E826F2AEC0BF00401740E826F1B
:1017E0002AEC0BF00401630E826F2AEC0BF004016B
:1017F000680E826F2AEC0BF074EF19F02F96CD0E65
:101800000C6E2FC00BF0E0EC08F0CD0EF7EC08F0FA
:10181000E8CF2FF02FB006D00401630E826F2AECC0
:101820000BF005D00401430E826F2AEC0BF02FB2AF
:1018300006D00401720E826F2AEC0BF005D0040171
:10184000520E826F2AEC0BF02FB406D00401670E03
:10185000826F2AEC0BF005D00401470E826F2AEC50
:101860000BF02FB606D00401740E826F2AEC0BF039
:1018700005D00401540E826F2AEC0BF074EF19F0BE
:101880000401410E826F2AEC0BF003018351310AEF
:10189000D8B4E4EF0EF003018351320AD8B414EF48
:1018A0000EF003018351330AD8B49DEF0DF003010C
:1018B0008351340AD8B48DEF0CF003018351350AFB
:1018C000D8B46AEF0CF004013F0E826F2AEC0BF0E3
:1018D00074EF19F004012C0E826F2AEC0BF0030157
:1018E0008451300AD8B47DEF0CF003018451310AE1
:1018F000D8B485EF0CF0D6EF0DF08B900401300ECC
:10190000826F2AEC0BF08BEF0CF08B800401310E10
:10191000826F2AEC0BF074EF19F0CC0EF7EC08F0A4
:10192000E8CF0BF004012C0E826F2AEC0BF00301C0
:101930008451310AD8B4B1EF0CF003018451300A5C
:10194000D8B4B3EF0CF0030184514D0AD8B4BDEF05
:101950000CF003018451540AD8B4C4EF0CF0DBEF4F
:101960000CF08A8401D08A940BAE04D00BAC02D068
:101970000BBA21D0E00E0B1218D01F0E0B168539B2
:10198000E844E00B0B1211D0E00E0B166BEC20F0CC
:1019900085C332F186C333F10101296B78EC20F065
:1019A000EFEC1FF000511F0B0B12CC0E0C6E0BC096
:1019B0000BF0E0EC08F00401340E826F2AEC0BF01F
:1019C00004012C0E826F2AEC0BF0CC0EF7EC08F021
:1019D000E8CF1AF08AB406D00401300E826F2AECE8
:1019E0000BF005D00401310E826F2AEC0BF00401DC
:1019F0002C0E826F2AEC0BF01A38E840070BE8CF68
:101A000082F40401300E82272AEC0BF004012C0E24
:101A1000826F2AEC0BF02AEC20F01A501F0BE8CF53
:101A200000F1CDEC1FF032C182F40401300E8227A8
:101A30002AEC0BF033C182F40401300E82272AEC29
:101A40000BF004012C0E826F2AEC0BF02AEC20F034
:101A50002DC000F100AF0BD0FF0E016FFF0E026F23
:101A6000FF0E036F04012D0E826F2AEC0BF0CDECFC
:101A70001FF031C182F40401300E82272AEC0BF0F2
:101A800032C182F40401300E82272AEC0BF033C1FC
:101A900082F40401300E82272AEC0BF004012C0E94
:101AA000826F2AEC0BF02AEC20F02CC000F1CDEC78
:101AB0001FF031C182F40401300E82272AEC0BF0B2
:101AC00032C182F40401300E82272AEC0BF033C1BC
:101AD00082F40401300E82272AEC0BF004012C0E54
:101AE000826F2AEC0BF02AEC20F02EC000F100AF40
:101AF0000BD0FF0E016FFF0E026FFF0E036F04018C
:101B00002D0E826F2AEC0BF0CDEC1FF031C182F468
:101B10000401300E82272AEC0BF032C182F404015A
:101B2000300E82272AEC0BF033C182F40401300E10
:101B300082272AEC0BF074EF19F0CB0EF7EC08F0CB
:101B4000E8CF0BF004012C0E826F2AEC0BF003019E
:101B50008451450AD8B4C1EF0DF003018451440A01
:101B6000D8B4C4EF0DF003018451300AD8B4C7EFE4
:101B70000DF003018451310AD8B4CBEF0DF0D6EF4C
:101B80000DF00B9ED0EF0DF00B8ED0EF0DF0FC0E94
:101B90000B16D0EF0DF0FC0E0B160B80D0EF0DF0F6
:101BA000CB0E0C6E0BC00BF0E0EC08F00401330E12
:101BB000826F2AEC0BF004012C0E826F2AEC0BF0E2
:101BC000CB0EF7EC08F0E8CF19F019BEEFEF0DF0EF
:101BD0000401450E826F2AEC0BF0F4EF0DF00401C6
:101BE000440E826F2AEC0BF004012C0E826F2AEC5B
:101BF0000BF00401300E826F2AEC0BF004012C0E66
:101C0000826F2AEC0BF019B00DEF0EF00401300ECC
:101C1000826F2AEC0BF012EF0EF00401310E826F8E
:101C20002AEC0BF074EF19F0CA0EF7EC08F0E8CFCD
:101C30000BF004012C0E826F2AEC0BF0030184518F
:101C4000450AD8B450EF0EF003018451440AD8B4C9
:101C500053EF0EF0030184514D0AD8B45CEF0EF03F
:101C600003018451410AD8B456EF0EF003018451A8
:101C7000460AD8B459EF0EF003018451560AD8B47D
:101C800064EF0EF003018451500AD8B46FEF0EF0E8
:101C900003018451520AD8B472EF0EF07BEF0EF0BC
:101CA0000B9E75EF0EF00B8E75EF0EF00B9C75EF23
:101CB0000EF00B8C75EF0EF0FC0E0B1685C3E8FFD3
:101CC000030B0B1275EF0EF0C70E0B1685C3E8FF62
:101CD000070BE846E846E8460B1275EF0EF00B845A
:101CE00075EF0EF00B9475EF0EF0CA0E0C6E0BC074
:101CF0000BF0E0EC08F0CA0EF7EC08F0E8CF18F0B3
:101D00000401320E826F2AEC0BF004012C0E826F5C
:101D10002AEC0BF018BE94EF0EF00401450E826F12
:101D20002AEC0BF099EF0EF00401440E826F2AECBE
:101D30000BF004012C0E826F2AEC0BF018C0E8FFA8
:101D4000030BE8CF82F40401300E82272AEC0BF05B
:101D500004012C0E826F2AEC0BF018BCB7EF0EF0CA
:101D60000401410E826F2AEC0BF0BCEF0EF004016F
:101D7000460E826F2AEC0BF004012C0E826F2AECC7
:101D80000BF018C0E8FF380BE842E842E842E8CF21
:101D900082F40401300E82272AEC0BF004012C0E91
:101DA000826F2AEC0BF018B4DDEF0EF00401520E36
:101DB000826F2AEC0BF0E2EF0EF00401500E826FFE
:101DC0002AEC0BF074EF19F0C90EF7EC08F0E8CF2D
:101DD0000BF004012C0E826F2AEC0BF003018451EE
:101DE000450AD8B402EF0FF003018451440AD8B475
:101DF00005EF0FF0030184514D0AD8B408EF0FF03E
:101E000016EF0FF00B9E10EF0FF00B8E10EF0FF090
:101E1000F80E0B1685C3E8FF070B0B1210EF0FF03F
:101E2000C90E0C6E0BC00BF0E0EC08F00401310E93
:101E3000826F2AEC0BF004012C0E826F2AEC0BF05F
:101E4000C90EF7EC08F0E8CF17F017BE06D0040172
:101E5000450E826F2AEC0BF005D00401440E826F10
:101E60002AEC0BF004012C0E826F2AEC0BF017C049
:101E7000E8FF070BE8CF82F40401300E82272AEC3A
:101E80000BF004012C0E826F2AEC0BF007802AEC79
:101E900020F028C0E8FF003B00430043030BCDECDB
:101EA0001FF033C182F40401300E82272AEC0BF0BC
:101EB00004012C0E826F2AEC0BF02AEC20F028C0D3
:101EC00001F1019F019D29C000F10101CDEC1FF03E
:101ED0002FC182F40401300E82272AEC0BF030C1AE
:101EE00082F40401300E82272AEC0BF031C182F417
:101EF0000401300E82272AEC0BF032C182F4040177
:101F0000300E82272AEC0BF033C182F40401300E2C
:101F100082272AEC0BF004012C0E826F2AEC0BF0C6
:101F20002AEC20F02AC001F12BC000F1D890013337
:101F30000033D890013300330101CDEC1FF02FC1E5
:101F400082F40401300E82272AEC0BF030C182F4B7
:101F50000401300E82272AEC0BF031C182F4040117
:101F6000300E82272AEC0BF032C182F40401300ECD
:101F700082272AEC0BF033C182F40401300E822751
:101F80002AEC0BF074EF19F0FC0EF7EC08F0E8CF38
:101F90000BF003018351520AD8B4FBEF0FF0030199
:101FA0008351720AD8B4FEEF0FF003018351500A37
:101FB000D8B401EF10F003018351700AD8B404EFD4
:101FC00010F003018351550AD8B407EF10F0030154
:101FD0008351750AD8B40AEF10F003018351430A04
:101FE000D8B413EF10F003018351630AD8B416EF8D
:101FF00010F01FEF10F00B9019EF10F00B8019EF9D
:1020000010F00B9219EF10F00B8219EF10F00B94F7
:1020100019EF10F00B8419EF10F00B9619EF10F078
:102020000B8619EF10F00B9819EF10F00B8819EFD1
:1020300010F0FC0E0C6E0BC00BF0E0EC08F004018D
:10204000590E826F2AEC0BF0119011921194119895
:10205000FC0EF7EC08F0E8CF0BF00BA011800BA200
:1020600011820BA411840BA8118811A03FEF10F06E
:102070000401520E826F2AEC0BF044EF10F00401C1
:10208000720E826F2AEC0BF011A84EEF10F00401D3
:10209000430E826F2AEC0BF053EF10F00401630E35
:1020A000826F2AEC0BF011A25DEF10F00401500ECC
:1020B000826F2AEC0BF062EF10F00401700E826F59
:1020C0002AEC0BF011A46CEF10F00401550E826F96
:1020D0002AEC0BF071EF10F00401750E826F2AEC00
:1020E0000BF074EF19F004016D0E826F2AEC0BF007
:1020F00003018351300AD8B4CBEF10F003018351B0
:10210000310AD8B4DEEF10F003018351320AD8B49B
:10211000F1EF10F076EF19F004014D0E826F2AEC0A
:102120000BF06BEC20F084C331F185C332F186C330
:1021300033F10101296B78EC20F0EFEC1FF0030183
:102140008351300AD8B4B3EF10F003018351310A40
:10215000D8B4BBEF10F003018351320AD8B4C3EFF7
:1021600010F076EF19F0FD0E0C6E00C10BF0E0ECF4
:1021700008F0CBEF10F0FE0E0C6E00C10BF0E0EC9F
:1021800008F0DEEF10F0FF0E0C6E00C10BF0E0EC7B
:1021900008F0F1EF10F00401300E826F2AEC0BF022
:1021A00004012C0E826F2AEC0BF02AEC20F0FD0EBD
:1021B000F7EC08F0E8CF00F102EF11F00401310E66
:1021C000826F2AEC0BF004012C0E826F2AEC0BF0CC
:1021D0002AEC20F0FE0EF7EC08F0E8CF00F102EF59
:1021E00011F00401320E826F2AEC0BF02AEC20F081
:1021F00004012C0E826F2AEC0BF0FF0EF7EC08F0B6
:10220000E8CF00F1CDEC1FF031C182F40401300EB3
:1022100082272AEC0BF032C182F40401300E8227AF
:102220002AEC0BF033C182F40401300E82272AEC31
:102230000BF074EF19F08351610AD8A476EF19F00E
:102240008451750AD8A476EF19F08551640AD8A490
:1022500076EF19F086C32AF187C32BF188C32CF1DE
:1022600089C32DF18AC32EF18BC32FF18CC330F1BA
:102270008DC331F18EC332F18FC333F10101296B6C
:1022800078EC20F0EFEC1FF000C1AFFF01C1B0FF10
:102290001E0E0C6EAFCF0BF0E0EC08F01F0E0C6EB4
:1022A000B0CF0BF0E0EC08F076EF19F080B660EFFD
:1022B00011F00401300E826F2AEC0BF065EF11F083
:1022C0000401310E826F2AEC0BF034EC0BF076EF48
:1022D00019F083C32AF184C32BF185C32CF186C383
:1022E0002DF187C32EF188C32FF189C330F18AC342
:1022F00031F18BC332F18CC333F1010178EC20F062
:10230000EFEC1FF0160E0C6E00C10BF0E0EC08F0C5
:10231000170E0C6E01C10BF0E0EC08F0180E0C6EFD
:1023200002C10BF0E0EC08F0190E0C6E03C10BF0CB
:10233000E0EC08F000C18AF101C18BF102C18CF11F
:1023400003C18DF100C18EF101C18FF102C190F185
:1023500003C191F14BEF12F083C32AF184C32BF137
:1023600085C32CF186C32DF187C32EF188C32FF1CD
:1023700089C330F18AC331F18BC332F18CC333F19D
:10238000010178EC20F0EFEC1FF000C18AF101C1EF
:102390008BF102C18CF103C18DF100C18EF101C13D
:1023A0008FF102C190F103C191F14BEF12F083C3A1
:1023B0002AF184C32BF185C32CF186C32DF187C389
:1023C0002EF188C32FF189C330F18AC331F18CC358
:1023D00032F18DC333F1010178EC20F0EFEC1FF006
:1023E0000101000E046F000E056F010E066F000E56
:1023F000076F40EC1FF01A0E0C6E00C10BF0E0EC02
:1024000008F01B0E0C6E01C10BF0E0EC08F01C0E86
:102410000C6E02C10BF0E0EC08F01D0E0C6E03C157
:102420000BF0E0EC08F000C192F101C193F102C1A0
:1024300094F103C195F14BEF12F083C32AF184C3E9
:102440002BF185C32CF186C32DF187C32EF188C3F0
:102450002FF189C330F18AC331F18CC332F18DC3BE
:1024600033F1010178EC20F0EFEC1FF00101000ED8
:10247000046F000E056F010E066F000E076F40EC33
:102480001FF000C192F101C193F102C194F103C1A7
:1024900095F14BEF12F0160EF7EC08F0E8CF00F1D3
:1024A000170EF7EC08F0E8CF01F1180EF7EC08F082
:1024B000E8CF02F1190EF7EC08F0E8CF03F1CDEC0C
:1024C0001FF090EC1DF00401730E826F2AEC0BF0EC
:1024D00004012C0E826F2AEC0BF08AC100F18BC133
:1024E00001F18CC102F18DC103F1CDEC1FF090EC34
:1024F0001DF00401730E826F2AEC0BF004012C0E08
:10250000826F2AEC0BF01A0EF7EC08F0E8CF00F11E
:102510001B0EF7EC08F0E8CF01F11C0EF7EC08F009
:10252000E8CF02F11D0EF7EC08F0E8CF03F191ECD3
:1025300019F004012C0E826F2AEC0BF092C100F10D
:1025400093C101F194C102F195C103F191EC19F02D
:1025500034EC0BF076EF19F00401690E826F2AEC6F
:102560000BF004012C0E826F2AEC0BF00101040E1B
:10257000006F000E016F000E026F000E036FCDECB6
:102580001FF02CC182F40401300E82272AEC0BF0DC
:102590002DC182F40401300E82272AEC0BF02EC1EB
:1025A00082F40401300E82272AEC0BF02FC182F452
:1025B0000401300E82272AEC0BF030C182F40401B2
:1025C000300E82272AEC0BF031C182F40401300E68
:1025D00082272AEC0BF032C182F40401300E8227EC
:1025E0002AEC0BF033C182F40401300E82272AEC6E
:1025F0000BF004012C0E826F2AEC0BF00101050E8A
:10260000006F000E016F000E026F000E036FCDEC25
:102610001FF02CC182F40401300E82272AEC0BF04B
:102620002DC182F40401300E82272AEC0BF02EC15A
:1026300082F40401300E82272AEC0BF02FC182F4C1
:102640000401300E82272AEC0BF030C182F4040121
:10265000300E82272AEC0BF031C182F40401300ED7
:1026600082272AEC0BF032C182F40401300E82275B
:102670002AEC0BF033C182F40401300E82272AECDD
:102680000BF004012C0E826F2AEC0BF00101380EC6
:10269000006F000E016F000E026F000E036FCDEC95
:1026A0001FF02CC182F40401300E82272AEC0BF0BB
:1026B0002DC182F40401300E82272AEC0BF02EC1CA
:1026C00082F40401300E82272AEC0BF02FC182F431
:1026D0000401300E82272AEC0BF030C182F4040191
:1026E000300E82272AEC0BF031C182F40401300E47
:1026F00082272AEC0BF032C182F40401300E8227CB
:102700002AEC0BF033C182F40401300E82272AEC4C
:102710000BF004012C0E826F2AEC0BF0200EF86EE9
:10272000F76AF66A04010900F5CF82F42AEC0BF08F
:102730000900F5CF82F42AEC0BF00900F5CF82F402
:102740002AEC0BF00900F5CF82F42AEC0BF009001B
:10275000F5CF82F42AEC0BF00900F5CF82F42AECD5
:102760000BF00900F5CF82F42AEC0BF00900F5CF4D
:1027700082F42AEC0BF034EC0BF076EF19F0835175
:10278000630AD8A474EF19F08451610AD8A474EFD5
:1027900019F085516C0AD8A474EF19F08651410ADA
:1027A0003FE08651440A1BE08651420AD8B423EF29
:1027B00014F08651350AD8B400EF1BF08651360A62
:1027C000D8B455EF1BF08651370AD8B4BEEF1BF0D2
:1027D0008651380AD8B41CEF1CF074EF19F0079832
:1027E000079A04017A0E826F2AEC0BF00401780E2E
:1027F000826F2AEC0BF00401640E826F2AEC0BF05E
:102800000401550E826F2AEC0BF00CEF14F004015A
:102810004C0E826F2AEC0BF034EC0BF076EF19F0D3
:102820000788079A04017A0E826F2AEC0BF00401E4
:10283000410E826F2AEC0BF00401610E826F2AECCC
:102840000BF000EF14F00798078A04017A0E826FEC
:102850002AEC0BF00401420E826F2AEC0BF004010B
:10286000610E826F2AEC0BF000EF14F00101666735
:1028700041EF14F0676741EF14F0686741EF14F01F
:10288000696715D04F674CEF14F050674CEF14F0A8
:1028900051674CEF14F052670AD00101000E006F2F
:1028A000000E016F000E026F000E036F120011B8D0
:1028B0000AD00101620E046F010E056F000E066F53
:1028C000000E076F09D00101A70E046F020E056FFD
:1028D000000E066F000E076F66C100F167C101F1BF
:1028E00068C102F169C103F12FEC1FF003BFE9EFEA
:1028F00014F0119A119C0101000E046FA80E056FCF
:10290000550E066F020E076F66C100F167C101F137
:1029100068C102F169C103F166C186F167C187F13F
:1029200068C188F169C189F12FEC1FF003BF0BD09A
:102930000101000E866FA80E876F550E886F020E7C
:10294000896F118A119C0E0EF7EC08F0E8CF18F190
:102950000F0EF7EC08F0E8CF19F1100EF7EC08F0C5
:10296000E8CF1AF1110EF7EC08F0E8CF1BF178EC84
:102970001EF086C104F187C105F188C106F189C145
:1029800007F12FEC1FF007823CEC1EF078EC1EF0F4
:1029900007923CEC1EF086C100F187C101F188C1AD
:1029A00002F189C103F107923CEC1EF0CC0E046FDA
:1029B000E00E056F870E066F050E076F2FEC1FF0F8
:1029C00000C118F101C119F102C11AF103C11BF1D3
:1029D0003BD0119C119A0101800E006F1A0E016FFD
:1029E000060E026F000E036F4FC104F150C105F1D6
:1029F00051C106F152C107F12FEC1FF003AF05D012
:102A00002AEC20F0118C119A12000E0EF7EC08F04F
:102A1000E8CF18F10F0EF7EC08F0E8CF19F1100E1F
:102A2000F7EC08F0E8CF1AF1110EF7EC08F0E8CF58
:102A30001BF14FC100F150C101F151C102F152C16E
:102A400003F107823CEC1EF018C100F119C101F13D
:102A50001AC102F11BC103F112000401730E826F4F
:102A60002AEC0BF004012C0E826F2AEC0BF0078489
:102A700062C166F163C167F164C168F165C169F162
:102A80004BC14FF14CC150F14DC151F14EC152F10A
:102A900057C159F158C15AF1079453EC15F034EC71
:102AA0000BF076EF19F066C100F167C101F168C162
:102AB00002F169C103F10101CDEC1FF090EC1DF0B2
:102AC0000401630E826F2AEC0BF004012C0E826F5E
:102AD0002AEC0BF04FC100F150C101F151C102F1DC
:102AE00052C103F10101CDEC1FF090EC1DF0040187
:102AF000660E826F2AEC0BF004012C0E826F2AEC1A
:102B00000BF02AEC20F059C100F15AC101F101018A
:102B1000CDEC1FF090EC1DF00401740E826F2AECD6
:102B20000BF0120010820401530E826F2AEC0BF09E
:102B300004012C0E826F2AEC0BF083C32AF184C3AC
:102B40002BF185C32CF186C32DF187C32EF188C3E9
:102B50002FF189C330F18AC331F18BC332F18CC3B9
:102B600033F1010178EC20F0EFEC1FF000C166F1C9
:102B700001C167F102C168F103C169F18EC32AF195
:102B80008FC32BF190C32CF191C32DF192C32EF181
:102B900093C32FF194C330F195C331F196C332F151
:102BA00097C333F1010178EC20F0EFEC1FF000C186
:102BB0004FF101C150F102C151F103C152F16BEC6F
:102BC00020F099C32FF19AC330F19BC331F19CC31C
:102BD00032F19DC333F1010178EC20F0EFEC1FF0EE
:102BE00000C159F101C15AF153EC15F004012C0E4A
:102BF000826F2AEC0BF00DEF16F0118E19A002D0A7
:102C000019AE108C18BE02D018A4108E0301825188
:102C1000520A02E10F8201D00F928251750A02E13D
:102C2000108401D010948251550A02E1108601D01F
:102C3000109611A003D011A401D01084078410B203
:102C40007BEF16F010A467EF16F0B6C166F1B7C1BE
:102C500067F1B8C168F1B9C169F1BAC16AF1BBC124
:102C60006BF1BCC16CF1BDC16DF1BEC16EF1BFC1F4
:102C70006FF1C0C170F1C1C171F1C2C172F1C3C1C4
:102C800073F1C4C174F1C5C175F1C6C176F1C7C194
:102C900077F1C8C178F1C9C179F1CAC17AF1CBC164
:102CA0007BF1CCC17CF1CDC17DF1CEC17EF1CFC134
:102CB0007FF1D0C180F1D1C181F1D2C182F1D3C104
:102CC00083F1D4C184F1D5C185F16FEF16F062C1F3
:102CD00066F163C167F164C168F165C169F14BC117
:102CE0004FF14CC150F14DC151F14EC152F157C19C
:102CF00059F158C15AF107940FA09DEF16F0010148
:102D000092678AEF16F093678AEF16F094678AEF5E
:102D100016F095678EEF16F09DEF16F036EC14F076
:102D200092C104F193C105F194C106F195C107F177
:102D30002FEC1FF003BF3AEF19F036EC14F001014D
:102D4000000E046F000E056F010E066F000E076F78
:102D500060EC1FF011A02AD011A228D0CDEC1FF0FA
:102D6000296701D005D004012D0E826F2AEC0BF0EB
:102D700030C182F40401300E82272AEC0BF031C1FD
:102D800082F40401300E82272AEC0BF032C182F467
:102D90000401300E82272AEC0BF033C182F40401C7
:102DA000300E82272AEC0BF034EC0BF012A8C5D0C1
:102DB00012981AC01BF01B3A1B42070E1B1600018B
:102DC0001B50000AD8B469EF17F000011B50010A2C
:102DD000D8B4F5EF16F000011B50020AD8B4F3EF97
:102DE00016F09BEF17F09BEF17F02AEC20F02AC0AB
:102DF00001F12BC000F1D89001330033D89001339A
:102E000000330101630E046F000E056F000E066FA4
:102E1000000E076F60EC1FF0280E046F000E056FA8
:102E2000000E066F000E076F2FEC1FF000C12DF093
:102E30002AEC20F028C001F1019F019D29C000F17A
:102E40000101A40E046F000E056F000E066F000E48
:102E5000076F60EC1FF000C12CF000C104F101C14C
:102E600005F102C106F103C107F1640E006F000E07
:102E7000016F000E026F000E036F2FEC1FF0050EA6
:102E8000046F000E056F000E066F000E076F60ECFA
:102E90001FF000C104F101C105F102C106F103C137
:102EA00007F12AEC20F02DC000F12FEC1FF000C13B
:102EB0002EF02EC0E8FF050F2D5C03E78A849BEF00
:102EC00017F02EC0E8FF0A0F2D5C01E68A949BEFF5
:102ED00017F000C124F101C125F102C126F103C19F
:102EE00027F12AEC20F030EC20F01A501F0BE8CF2D
:102EF00000F10101640E046F000E056F000E066FF5
:102F0000000E076F40EC1FF024C104F125C105F14C
:102F100026C106F127C107F12FEC1FF003BF02D035
:102F20008A9401D08A8424C100F125C101F126C10F
:102F300002F127C103F176EF19F000C124F101C1BC
:102F400025F102C126F103C127F110AE4DD0109E2C
:102F500000C108F101C109F102C10AF103C10BF17D
:102F6000CDEC1FF030C1D6F131C1D7F132C1D8F16B
:102F700033C1D9F108C100F109C101F10AC102F15F
:102F80000BC103F101016C0E046F070E056F000EFB
:102F9000066F000E076F2FEC1FF003BF04D0010176
:102FA000550EDA6F1CD008C100F109C101F10AC148
:102FB00002F10BC103F10101A40E046F060E056FAF
:102FC000000E066F000E076F2FEC1FF003BF04D03A
:102FD00001017F0EDA6F03D00101FF0EDA6F1C8E44
:102FE00011AE3AEF19F0119E24C100F125C101F193
:102FF00026C102F127C103F111A005D011A203D00F
:103000000FB03AEF19F010A40DEF18F00401750E8F
:10301000826F2AEC0BF012EF18F00401720E826F2F
:103020002AEC0BF004012C0E826F2AEC0BF0CDEC95
:103030001FF0296721EF18F00401200E826F24EFA2
:1030400018F004012D0E826F2AEC0BF030C182F4CF
:103050000401300E82272AEC0BF031C182F4040106
:10306000300E82272AEC0BF004012E0E826F2AEC20
:103070000BF032C182F40401300E82272AEC0BF0EF
:1030800033C182F40401300E82272AEC0BF00401D4
:103090006D0E826F2AEC0BF004012C0E826F2AEC6D
:1030A0000BF04FC100F150C101F151C102F152C109
:1030B00003F10101CDEC1FF090EC1DF00401480E6E
:1030C000826F2AEC0BF004017A0E826F2AEC0BF06F
:1030D00004012C0E826F2AEC0BF066C100F167C16F
:1030E00001F168C102F169C103F10101CDEC1FF0EA
:1030F00090EC1DF00401630E826F2AEC0BF00401CA
:103100002C0E826F2AEC0BF066C100F167C101F151
:1031100068C102F169C103F101010A0E046F000EDA
:10312000056F000E066F000E076F40EC1FF0000EDB
:10313000046F120E056F000E066F000E076F60EC35
:103140001FF0CDEC1FF02AC182F40401300E82275B
:103150002AEC0BF02BC182F40401300E82272AECFA
:103160000BF02CC182F40401300E82272AEC0BF004
:103170002DC182F40401300E82272AEC0BF02EC1FF
:1031800082F40401300E82272AEC0BF02FC182F466
:103190000401300E82272AEC0BF030C182F40401C6
:1031A000300E82272AEC0BF004012E0E826F2AECDF
:1031B0000BF031C182F40401300E82272AEC0BF0AF
:1031C00032C182F40401300E82272AEC0BF033C1A5
:1031D00082F40401300E82272AEC0BF00401730EF6
:1031E000826F2AEC0BF004012C0E826F2AEC0BF09C
:1031F0002AEC20F059C100F15AC101F1A0EC1AF0FB
:103200000FB206EF19F00FA038EF19F004012C0EE1
:10321000826F2AEC0BF0200EF86EF76AF66A040152
:103220000900F5CF82F42AEC0BF00900F5CF82F407
:103230002AEC0BF00900F5CF82F42AEC0BF0090020
:10324000F5CF82F42AEC0BF00900F5CF82F42AECDA
:103250000BF00900F5CF82F42AEC0BF00900F5CF52
:1032600082F42AEC0BF00900F5CF82F42AEC0BF083
:1032700034EC0BF00F90109E129876EF19F00401C9
:10328000630E826F2AEC0BF004012C0E826F2AEC85
:103290000BF07CEC19F004012C0E826F2AEC0BF081
:1032A000EFEC19F004012C0E826F2AEC0BF06BECA2
:1032B0001AF004012C0E826F2AEC0BF00101F80EBB
:1032C000006FCD0E016F660E026F030E036F91EC5F
:1032D00019F004012C0E826F2AEC0BF081EC1AF02D
:1032E00034EC0BF076EF19F034EC0BF00301C26B09
:1032F0000790109285EF1CF0D8900E0EF7EC08F0B6
:10330000E8CF00F10F0EF7EC08F0E8CF01F1100E56
:10331000F7EC08F0E8CF02F1110EF7EC08F0E8CF77
:1033200003F10101000E046F000E056F010E066F20
:10333000000E076F60EC1FF0CDEC1FF02AC182F485
:103340000401300E82272AEC0BF02BC182F4040119
:10335000300E82272AEC0BF02CC182F40401300ECF
:1033600082272AEC0BF02DC182F40401300E822753
:103370002AEC0BF02EC182F40401300E82272AECD5
:103380000BF02FC182F40401300E82272AEC0BF0DF
:1033900030C182F40401300E82272AEC0BF031C1D7
:1033A00082F40401300E82272AEC0BF004012E0E69
:1033B000826F2AEC0BF032C182F40401300E8227B6
:1033C0002AEC0BF033C182F40401300E82272AEC80
:1033D0000BF004016D0E826F2AEC0BF01200120E3E
:1033E000F7EC08F0E8CF00F1130EF7EC08F0E8CFA7
:1033F00001F1140EF7EC08F0E8CF02F1150EF7EC2E
:1034000008F0E8CF03F101010A0E046F000E056F0A
:10341000000E066F000E076F40EC1FF0000E046FE9
:10342000120E056F000E066F000E076F60EC1FF0A6
:10343000CDEC1FF02AC182F40401300E82272AEC61
:103440000BF02BC182F40401300E82272AEC0BF022
:103450002CC182F40401300E82272AEC0BF02DC11E
:1034600082F40401300E82272AEC0BF02EC182F484
:103470000401300E82272AEC0BF02FC182F40401E4
:10348000300E82272AEC0BF030C182F40401300E9A
:1034900082272AEC0BF004012E0E826F2AEC0BF02F
:1034A00031C182F40401300E82272AEC0BF032C1C4
:1034B00082F40401300E82272AEC0BF033C182F42F
:1034C0000401300E82272AEC0BF00401730E826F88
:1034D0002AEC0BF012000A0EF7EC08F0E8CF00F12E
:1034E0000B0EF7EC08F0E8CF01F10C0EF7EC08F04A
:1034F000E8CF02F10D0EF7EC08F0E8CF03F1A0EFF2
:103500001AF0060EF7EC08F0E8CF00F1070EF7EC22
:1035100008F0E8CF01F1080EF7EC08F0E8CF02F16F
:10352000090EF7EC08F0E8CF03F1A0EF1AF0010163
:103530002AEC20F0078457C100F158C101F107942B
:103540000101E80E046F800E056F000E066F000E7D
:10355000076F40EC1FF0000E046F040E056F000EA5
:10356000066F000E076F60EC1FF0880E046F130EDD
:10357000056F000E066F000E076F2FEC1FF00A0E8E
:10358000046F000E056F000E066F000E076F60ECF3
:103590001FF0CDEC1FF001012967D4EF1AF00401F0
:1035A000200E826FD7EF1AF004012D0E826F2AECE5
:1035B0000BF030C182F40401300E82272AEC0BF0AC
:1035C00031C182F40401300E82272AEC0BF032C1A3
:1035D00082F40401300E82272AEC0BF004012E0E37
:1035E000826F2AEC0BF033C182F40401300E822783
:1035F0002AEC0BF00401430E826F2AEC0BF0120050
:1036000087C32AF188C32BF189C32CF18AC32DF11A
:103610008BC32EF18CC32FF18DC330F18EC331F1EA
:1036200090C332F191C333F10101296B78EC20F0A2
:10363000EFEC1FF00101000E046F000E056F010E8C
:10364000066F000E076F40EC1FF00E0E0C6E00C1EF
:103650000BF0E0EC08F00F0E0C6E01C10BF0E0EC8B
:1036600008F0100E0C6E02C10BF0E0EC08F0110E29
:103670000C6E03C10BF0E0EC08F004017A0E826FCF
:103680002AEC0BF004012C0E826F2AEC0BF00401E3
:10369000350E826F2AEC0BF004012C0E826F2AEC9F
:1036A0000BF07CEC19F00CEF14F087C32AF188C3FF
:1036B0002BF189C32CF18AC32DF18BC32EF18CC35E
:1036C0002FF18DC330F18EC331F190C332F191C32C
:1036D00033F10101296B78EC20F0EFEC1FF0880E3C
:1036E000046F130E056F000E066F000E076F34ECAB
:1036F0001FF0000E046F040E056F000E066F000E23
:10370000076F40EC1FF00101E80E046F800E056F9B
:10371000000E066F000E076F60EC1FF00A0E0C6EB5
:1037200000C10BF0E0EC08F00B0E0C6E01C10BF0C9
:10373000E0EC08F00C0E0C6E02C10BF0E0EC08F0AF
:103740000D0E0C6E03C10BF0E0EC08F004017A0ED4
:10375000826F2AEC0BF004012C0E826F2AEC0BF026
:103760000401360E826F2AEC0BF004012C0E826FDE
:103770002AEC0BF06BEC1AF00CEF14F087C32AF173
:1037800088C32BF189C32CF18AC32DF18BC32EF191
:103790008CC32FF18DC330F18FC331F190C332F15F
:1037A00091C333F1010178EC20F0EFEC1FF0000E33
:1037B000046F120E056F000E066F000E076F40ECCF
:1037C0001FF001010A0E046F000E056F000E066F58
:1037D000000E076F60EC1FF0120E0C6E00C10BF0B4
:1037E000E0EC08F0130E0C6E01C10BF0E0EC08F0F9
:1037F000140E0C6E02C10BF0E0EC08F0150E0C6E0E
:1038000003C10BF0E0EC08F004017A0E826F2AECA1
:103810000BF004012C0E826F2AEC0BF00401370E22
:10382000826F2AEC0BF004012C0E826F2AEC0BF055
:10383000EFEC19F00CEF14F087C32AF188C32BF1D9
:1038400089C32CF18AC32DF18BC32EF18CC32FF1C8
:103850008DC330F18EC331F190C332F191C333F196
:103860000101296B78EC20F0EFEC1FF0880E046F5B
:10387000130E056F000E066F000E076F34EC1FF07D
:10388000000E046F040E056F000E066F000E076F2A
:1038900040EC1FF00101E80E046F800E056F000E72
:1038A000066F000E076F60EC1FF0060E0C6E00C175
:1038B0000BF0E0EC08F0070E0C6E01C10BF0E0EC31
:1038C00008F0080E0C6E02C10BF0E0EC08F0090ED7
:1038D0000C6E03C10BF0E0EC08F004017A0E826F6D
:1038E0002AEC0BF004012C0E826F2AEC0BF0040181
:1038F000380E826F2AEC0BF004012C0E826F2AEC3A
:103900000BF081EC1AF00CEF14F007A8F8EF1CF0A4
:103910000101800E006F1A0E016F060E026F000E7D
:10392000036F4BC104F14CC105F14DC106F14EC10D
:1039300007F12FEC1FF003BF3EEF1DF08AEC1DF0E6
:103940004BC100F14CC101F14DC102F14EC103F177
:1039500007823CEC1EF018C104F119C105F11AC12F
:1039600006F11BC107F1F80E006FCD0E016F660E58
:10397000026F030E036F2FEC1FF00E0E0C6E00C1D2
:103980000BF0E0EC08F00F0E0C6E01C10BF0E0EC58
:1039900008F0100E0C6E02C10BF0E0EC08F0110EF6
:1039A0000C6E03C10BF0E0EC08F0078401012AEC77
:1039B00020F057C100F158C101F107940A0E0C6EB6
:1039C00000C10BF0E0EC08F00B0E0C6E01C10BF027
:1039D000E0EC08F00C0E0C6E02C10BF0E0EC08F00D
:1039E0000D0E0C6E03C10BF0E0EC08F03EEF1DF085
:1039F00007AA3EEF1DF0078401012AEC20F057C111
:103A000000F158C101F10794060E0C6E00C10BF0D5
:103A1000E0EC08F0070E0C6E01C10BF0E0EC08F0D2
:103A2000080E0C6E02C10BF0E0EC08F0090E0C6EF3
:103A300003C10BF0E0EC08F0078462C100F163C140
:103A400001F164C102F165C103F10794120E0C6E1D
:103A500000C10BF0E0EC08F0130E0C6E01C10BF08E
:103A6000E0EC08F0140E0C6E02C10BF0E0EC08F074
:103A7000150E0C6E03C10BF0E0EC08F00798079AE6
:103A80000401805181197F0B0DE09EA8FED714EE32
:103A900000F081517F0BE126E750812B0F01AD6EC5
:103AA00040EF1DF077EF0AF018C100F119C101F1E4
:103AB0001AC102F11BC103F1000E046F000E056F65
:103AC000010E066F000E076F60EC1FF029A17FEF5B
:103AD0001DF02051D8B47FEF1DF018C100F119C1BD
:103AE00001F11AC102F11BC103F1000E046F000EB7
:103AF000056F0A0E066F000E076F60EC1FF01200D4
:103B0000010104510013055101130651021307511D
:103B1000031312000101186B196B1A6B1B6B120057
:103B20002AC182F40401300E82272AEC0BF02BC14B
:103B300082F40401300E82272AEC0BF02CC182F4AF
:103B40000401300E82272AEC0BF02DC182F404010F
:103B5000300E82272AEC0BF02EC182F40401300EC5
:103B600082272AEC0BF02FC182F40401300E822749
:103B70002AEC0BF030C182F40401300E82272AECCB
:103B80000BF031C182F40401300E82272AEC0BF0D5
:103B900032C182F40401300E82272AEC0BF033C1CB
:103BA00082F40401300E82272AEC0BF012002FC1A0
:103BB00082F40401300E82272AEC0BF030C182F42B
:103BC0000401300E82272AEC0BF031C182F404018B
:103BD000300E82272AEC0BF032C182F40401300E41
:103BE00082272AEC0BF033C182F40401300E8227C5
:103BF0002AEC0BF01200060E1E6E060E1F6E060E4D
:103C0000206E1E2E01EF1EF01F2E01EF1EF0202E43
:103C100001EF1EF08B84020E1E6E020E1F6E020E4E
:103C2000206E1E2E11EF1EF01F2E11EF1EF0202E03
:103C300011EF1EF08B941200FF0E1F6E1FC020F0BC
:103C4000030E1E6E8B841E2E22EF1EF0030E1E6EC0
:103C5000202E22EF1EF08B941FC020F0030E1E6E4C
:103C60001E2E30EF1EF0030E1E6E203E30EF1EF0B3
:103C70001F2E1EEF1EF012000101005305E101533B
:103C800003E1025301E1002BFFEC1EF02AEC20F0CF
:103C90003951006F3A51016F420E046F4B0E056FA0
:103CA000000E066F000E076F40EC1FF000C104F11C
:103CB00001C105F102C106F103C107F118C100F10C
:103CC00019C101F11AC102F11BC103F107B26DEF75
:103CD0001EF034EC1FF06FEF1EF02FEC1FF000C150
:103CE00018F101C119F102C11AF103C11BF112004F
:103CF0002AEC20F059C100F15AC101F1060EF7EC8F
:103D000008F0E8CF04F1070EF7EC08F0E8CF05F172
:103D1000080EF7EC08F0E8CF06F1090EF7EC08F012
:103D2000E8CF07F12FEC1FF000C124F101C125F10C
:103D300002C126F103C127F1290E046F000E056FA1
:103D4000000E066F000E076F40EC1FF0EE0E046FC2
:103D5000430E056F000E066F000E076F34EC1FF068
:103D600024C104F125C105F126C106F127C107F1DF
:103D700040EC1FF000C11CF101C11DF102C11EF198
:103D800003C11FF1120EF7EC08F0E8CF04F1130E97
:103D9000F7EC08F0E8CF05F1140EF7EC08F0E8CFE7
:103DA00006F1150EF7EC08F0E8CF07F10D0E006FE5
:103DB000000E016F000E026F000E036F40EC1FF04B
:103DC000180E046F000E056F000E066F000E076FD1
:103DD00060EC1FF01CC104F11DC105F11EC106F10C
:103DE0001FC107F134EC1FF06A0E046F2A0E056F35
:103DF000000E066F000E076F2FEC1FF01200BF0EB3
:103E0000FA6E200E3A6F396BD890003701370237BF
:103E10000337D8B010EF1FF03A2F05EF1FF0390726
:103E20003A070353D8B412000331070B80093F6FE0
:103E300003390F0B010F396F80EC5FF0406F3905CC
:103E400080EC5FF0405D405F396B3F33D8B039277D
:103E500039333FA925EF1FF04051392712000101E6
:103E60004FEC20F0D8B01200010103510719346F54
:103E700012EC20F0D8900751031934AF800F1200D4
:103E80000101346B36EC20F0D8A04CEC20F0D8B017
:103E9000120021EC20F02AEC20F01F0E366F62ECAD
:103EA00020F00B35D8B012EC20F0D8A00335D8B0F4
:103EB0001200362F4FEF1FF034B139EC20F0120012
:103EC0000101346B04510511061107110008D8A037
:103ED00036EC20F0D8A04CEC20F0D8B01200086BE3
:103EE000096B0A6B0B6B62EC20F01F0E366F62ECF5
:103EF00020F007510B5DD8A48AEF1FF006510A5D30
:103F0000D8A48AEF1FF00551095DD8A48AEF1FF0ED
:103F10000451085DD8A09DEF1FF00451085F0551C2
:103F2000D8A0053D095F0651D8A0063D0A5F07519C
:103F3000D8A0073D0B5FD8900081362F77EF1FF098
:103F400034B139EC20F0346B36EC20F0D89066ECCC
:103F500020F007510B5DD8A4BAEF1FF006510A5D9F
:103F6000D8A4BAEF1FF00551095DD8A4BAEF1FF02D
:103F70000451085DD8A0C9EF1FF0003FC9EF1FF042
:103F8000013FC9EF1FF0023FC9EF1FF0032BD8B468
:103F9000120034B139EC20F012000101346B36EC20
:103FA00020F0D8B012006BEC20F0200E366F0037F6
:103FB00001370237033711EE33F00A0E376FE73659
:103FC0000A0EE75CD8B0E76EE552372FDFEF1FF03F
:103FD000362FD7EF1FF034B12981D890120001019C
:103FE0000A0E346F200E366F11EE29F03451376F00
:103FF0000A0ED890E652D8B0E726E732372FFAEF0C
:104000001FF00333023301330033362FF4EF1FF078
:10401000E750FF0FD8A00335D8B0120029B139EC12
:1040200020F01200045100270551D8B0053D0127AA
:104030000651D8B0063D02270751D8B0073D0327E7
:1040400012000051086F0151096F02510A6F0351AC
:104050000B6F12000101006B016B026B036B12000E
:104060000101046B056B066B076B12000335D8A0CA
:1040700012000351800B001F011F021F031F003F8E
:1040800049EF20F0013F49EF20F0023F49EF20F0D7
:10409000032B342B032512000735D8A0120007513B
:1040A000800B041F051F061F071F043F5FEF20F052
:1040B000053F5FEF20F0063F5FEF20F0072B342B2A
:1040C0000725120000370137023703370837093751
:1040D0000A370B3712000101296B2A6B2B6B2C6BF3
:1040E0002D6B2E6B2F6B306B316B326B336B120081
:1040F00001012A510F0B2A6F2B510F0B2B6F2C51E3
:104100000F0B2C6F2D510F0B2D6F2E510F0B2E6F90
:104110002F510F0B2F6F30510F0B306F31510F0B91
:10412000316F32510F0B326F33510F0B336F12005F
:10BF0000E844F926000C160C2B0C3F0C520C640C68
:10BF1000760C860C960CA50CB30CC10CCF0CDC0C6B
:06BF2000E80CF40C000C1B
:00000001FF
